:020000040800F2
:100000003824002011200008192000081B200008B7
:100010001D2000081F20000821200008000000000B
:100020000000000000000000000000002320000885
:10003000252000080000000027200008B320000849
:100040002B2000082B2000082B2000082B20000864
:100050002B2000082B2000082B2000082B20000854
:100060002B2000082B2000082B2000082B20000844
:100070002B2000082B2000082B2000082B20000834
:100080002B2000082B2000082B2000082B20000824
:100090002B2000082B2000082B2000082B20000814
:1000A0002B2000082B2000082B200008ED22000840
:1000B0002B2000082B2000082B2000082B200008F4
:1000C0002B2000082B2000082B2000082B200008E4
:1000D0002B2000082B200008853200082B20000868
:1000E0002B2000082B2000082B2000080000000017
:1000F0000000000000000000000000000000000000
:1001000000000000000000002B2000082B20000849
:100110002B2000082B200008312C00082B20000881
:100120002B2000082B2000082B2000082B20000883
:100130002B2000082B2000082B2000082B20000873
:100140002B2000082B2000082B2000082B20000863
:1001500000F002F800F05EF80AA090E8000C82447B
:100160008344AAF10107DA4501D100F053F8AFF258
:10017000090EBAE80F0013F0010F18BFFB1A43F085
:10018000010318472C4B00004C4B000010F8013BBA
:100190000A4413F0030408BF10F8014B1D1108BFF7
:1001A00010F8015B641E05D010F8016B641E01F8A5
:1001B000016BF9D1002D15D010F8014B03F00C03A1
:1001C0000C2BA1EB04040ABF10F8013BA4EB831431
:1001D000A4EB032405F1010314F8016B5B1E01F885
:1001E000016BF9D5914238BF10F8013BD1D370476C
:1001F0000023002400250026103A28BF78C1FBD830
:10020000520728BF30C148BF0B6070471FB51FBDE4
:1002100010B510BD04F0F1FC1146FFF7F7FF03F035
:100220000DFF04F00FFD03B4FFF7F2FF03BC04F071
:1002300017FD000031490143314A1160704770B524
:10024000002100230F22C47804B32D4C246804F449
:10025000E064C4F5E064210AC1F10403CA404478B3
:1002600004FA03F18478144021430901254C0678EF
:10027000A155047804F01F050124AC4005786D11E8
:10028000AD0005F1E025C5F8004109E0047804F06F
:100290001F050124AC401C4D0678761145F8264018
:1002A00070BD1A4A0A400243154B1B1F1A60704763
:1002B00039B1134A121D12680243114B1B1D1A60FB
:1002C00006E00F4A121D126882430D4B1B1D1A6077
:1002D0007047042808D14FF0E021096941F004017A
:1002E0004FF0E022116107E04FF0E021096921F0B1
:1002F00004014FF0E0221161704700000000FA0590
:100300000CED00E000E400E080E100E080FFFF1F72
:1003100010B50446CC48844208D10121042000F0E5
:10032000E7FB0021042000F0E3FB46E0C7488442DD
:1003300008D10121082000F0DBFB0021082000F09B
:10034000D7FB3AE0C248844208D10121102000F0D6
:10035000CFFB0021102000F0CBFB2EE0BD488442F3
:1003600008D10121202000F0C3FB0021202000F053
:10037000BFFB22E0B848844208D10121402000F0B0
:10038000B7FB0021402000F0B3FB16E0B3488442E5
:1003900008D10121802000F0ABFB0021802000F07B
:1003A000A7FB0AE0AE48844207D10121801500F086
:1003B0009FFB0021A01500F09BFB10BD10B5012193
:1003C000084600F095FB0021012000F091FB10BDD4
:1003D0002DE9F041024600250026002000230024DC
:1003E000002791F803C00CF00F0591F803C00CF042
:1003F000100CBCF1000F03D091F802C04CEA0505C7
:1004000091F800C0BCF1000F31D0146800202BE03F
:100410004FF0010C0CFA00F3B1F800C00CEA03062F
:100420009E4220D183004FF00F0C0CFA03F7BC431F
:1004300005FA03FC4CEA040491F803C0BCF1280F50
:1004400006D14FF0010C0CFA00FCC2F814C00AE00F
:1004500091F803C0BCF1480F05D14FF0010C0CFA24
:1004600000FCC2F810C0401C0828D1D31460B1F8B9
:1004700000C0BCF1FF0F34DD546800202EE000F115
:10048000080C4FF0010808FA0CF3B1F800C00CEAB0
:1004900003069E4221D183004FF00F0C0CFA03F7A4
:1004A000BC4305FA03FC4CEA040491F803C0BCF118
:1004B000280F05D100F1080C08FA0CF8C2F81480D6
:1004C00091F803C0BCF1480F07D100F1080C4FF0C0
:1004D000010808FA0CF8C2F81080401C0828CED396
:1004E0005460BDE8F0814FF6FF71018002218170F8
:1004F0000421C17070470246002093680B400BB185
:10050000012000E0002070470146886880B27047F3
:1005100002460020D3680B400BB1012000E0002010
:1005200070470146C86880B27047016170474161F9
:1005300070470AB1016100E041617047C1607047D6
:100540004FF480320A4382618161826182698269EB
:10055000704702460020434B18684FF680731840DE
:1005600040EA021008433F4B186070473E49C8619B
:100570007047F0B50A46002300240021002500F052
:100580000046B6F1004F02D1364EF16901E0354E1A
:100590007168C0F3034583B200F44016B6F5401FFE
:1005A00008D121F070612F4E766826F070662D4FCD
:1005B0007E6012E000F48016B6F5801F06D1032697
:1005C00006FA05F4A14341F0706106E0460D3601DC
:1005D00003FA06F6B14341F0706122B1460D3601CF
:1005E00003FA06F6314300F00046B6F1004F02D19F
:1005F0001C4EF16101E01B4E7160F0BD30B5002270
:100600008B071C0F0F2303FA04F2164B08338C10D0
:1006100053F824309343134C08348D1044F825309C
:1006200023468C1053F824308C07240F00FA04F46E
:1006300023430C4C08348D1044F8253030BD0A4952
:10064000DC3108607047000000080140000C0140E8
:10065000001001400014014000180140001C01403E
:10066000002001400000014000002042FB480068DB
:1006700040F00100F949086008464068F849084020
:10068000F649486008460068F6490840F3490860A2
:100690000846006820F4802008600846406820F47E
:1006A000FE0048600846006820F0A05008604FF443
:1006B0007F0088600020C8627047E849096821F41B
:1006C0008031E64A11601146096821F480211160E9
:1006D000B0F5803F03D0B0F5802F0ED106E0DF49A2
:1006E000096841F48031DD4A116007E0DB4909689F
:1006F00041F4A021D94A116000E000BF00BF70475B
:1007000010B501460022002300204A11012A02D11F
:10071000D24C236806E0022A02D1D04C236A01E0C1
:10072000CE4C636A01F01F02012494401C400CB1BE
:10073000012000E0002010BD38B50020009000240A
:10074000002500BF3120FFF7DBFF05460098401C65
:1007500000900098B0F5A06F01D0002DF2D03120AC
:10076000FFF7CEFF08B1012400E00024204638BD89
:1007700001460020B94A106820F0F80040EAC100A4
:1007800010607047B8490860704702460020B34BBC
:10079000586820F4741042EA01031843AF4B5860C4
:1007A0007047B1490866704702460020AB4BD86AD3
:1007B000AE4B184042EA01031843A84BD862704779
:1007C00001460020A54AD06A20F0F0000843D0621C
:1007D000704701460020A14AD06A20F470600843A7
:1007E000D0627047A04988667047014600209B4A46
:1007F000D06A20F470400843D06270479A49086775
:10080000704701460020954A506820F003000843D5
:10081000506070479148406800F00C0070470146F6
:1008200000208E4A506820F0F00008435060704766
:1008300001460020894A506820F4E0600843506077
:10084000704701460020854A506820F4605040EA15
:10085000C1005060704729B1804A527A02437F4BF1
:100860005A7204E07D4A527A82437C4B5A72704736
:100870007D49D8310860704701460020774A5068AA
:1008800020F4404008435060704779490860704741
:100890007749091D086070470021704A20321170A5
:1008A0006E4A82F82010012802D004280AD104E000
:1008B00001216A4A2032117005E00521674A203281
:1008C000117000E000BF00BF70476A4908607047C0
:1008D0006249096A0143614A1162704765494439B6
:1008E000086070472DE9F041002100220025002317
:1008F0000026002400278C46DFF86081D8F80480A9
:1009000008F00C0121B1042907D0082959D109E0C8
:10091000DFF86481C0F8008058E0DFF85C81C0F83F
:10092000008053E0DFF83481D8F8048008F47012B6
:10093000DFF82881D8F8048008F48035920C0D2A5D
:1009400001D0921C00E0062235B9DFF8308102FBAD
:1009500008F8C0F8008033E0DFF80081D8F82C8078
:1009600008F48036DFF8F480D8F82C8008F00F08FF
:1009700008F1010446B9DFF80081B8FBF4F808FB80
:1009800002F8C0F800801BE0DFF8D080D8F82C8097
:10099000C8F3031808F10107DFF8C080D8F82C80ED
:1009A000C8F3032808F1020CDFF8CC80B8FBF7F895
:1009B00008FB0CF8B8FBF4F808FB02F8C0F800805C
:1009C00004E0DFF8B480C0F8008000BF00BFDFF8AB
:1009D0008C80D8F8048008F0F0010909DFF8A080C5
:1009E00018F80130D0F8008028FA03F8C0F8048025
:1009F000DFF86880D8F8048008F4E061090ADFF8BD
:100A0000808018F80130D0F8048028FA03F8C0F884
:100A10000880DFF84880D8F8048008F46051C90ADB
:100A2000DFF85C8018F80130D0F8048028FA03F869
:100A3000C0F80C80DFF82480D8F8048008F4404126
:100A4000890BDFF8408018F80130D0F80C80B8FB33
:100A5000F3F8C0F81080BDE8F081000000100240FB
:100A60000000FFF0FFFFF6FE00004242F0FFFEFF35
:100A7000C40542428004424200127A0000093D004F
:100A8000000000201000002029B1354A52690243BD
:100A9000334B5A6104E0324A52698243304B5A6107
:100AA000704729B12E4A926902432D4B9A6104E0A6
:100AB0002B4A926982432A4B9A61704729B1284A8E
:100AC000D2690243264BDA6104E0254AD2698243A7
:100AD000234BDA61704729B1214A926A0243204BC5
:100AE0009A6204E01E4A926A82431D4B9A627047E2
:100AF00029B11B4AD2680243194BDA6004E0184A54
:100B0000D2688243164BDA60704729B1144A1269E1
:100B10000243134B1A6104E0114A12698243104BDD
:100B20001A6170470F49086070470F49C8647047E1
:100B30000B49C87170470A48406A40F08070084904
:100B40004862704701460020054A92680A400AB18F
:100B5000012000E0002070470149887270470000C2
:100B600000100240400442420000424210B50446D8
:100B7000FE48844208D10121C014FFF7B9FF0021CB
:100B8000E014FFF7B5FFC4E0B4F1804F08D10121B4
:100B90000846FFF7BAFF00210120FFF7B6FFB8E0D3
:100BA000F348844208D101210220FFF7AEFF002163
:100BB0000220FFF7AAFFACE0EE48844208D10121F1
:100BC0000420FFF7A2FF00210420FFF79EFFA0E012
:100BD000E948844208D101210820FFF796FF00214F
:100BE0000820FFF792FF94E0E448844208D10121F5
:100BF0001020FFF78AFF00211020FFF786FF88E012
:100C0000DF48844208D101212020FFF77EFF002128
:100C10002020FFF77AFF7CE0DA48844208D10121E6
:100C20004014FFF765FF00216014FFF761FF70E0DB
:100C3000D548844209D10121C804FFF759FF00219A
:100C40004FF40020FFF754FF63E0D048844209D1FD
:100C500001210805FFF74CFF00214FF48010FFF73A
:100C600047FF56E0CA48844209D101214805FFF7F1
:100C70003FFF00214FF40010FFF73AFF49E0C5485D
:100C8000844208D101214020FFF73FFF002140208E
:100C9000FFF73BFF3DE0C048844208D1012180209E
:100CA000FFF733FF00218020FFF72FFF31E0BB4823
:100CB000844208D101218015FFF727FF0021A015EC
:100CC000FFF723FF25E0B648844209D1012108043B
:100CD000FFF70EFF00214FF48030FFF709FF18E007
:100CE000B048844209D101214804FFF701FF0021E7
:100CF0004FF40030FFF7FCFE0BE0AB48844208D114
:100D000001218804FFF7F4FE00214FF48020FFF753
:100D1000EFFE10BD00220288944B98420ED0994BF2
:100D200098420BD0B0F1804F08D0914B984205D03B
:100D3000904B984202D0904B984204D14FF68F735B
:100D40001A404B881A438D4B984207D08C4B9842DF
:100D500004D04FF6FF431A40CB881A4302808B8899
:100D600083850B880385814B98420BD0854B984235
:100D700008D08B4B984205D08A4B984202D08A4BC0
:100D8000984201D10B7A038601238382704770B5A4
:100D9000002400220023058C4FF6FE7635400584A2
:100DA000028C8388048B4FF68F752C40B51E2C4027
:100DB0000D882C43751E2A400D892A434D882A43ED
:100DC0006A4DA8420BD06F4DA84208D0744DA8427E
:100DD00005D0744DA84202D0734DA84213D14FF6EE
:100DE000F7752A404D892A434FF6FB752A408D88B6
:100DF0002A434FF6FF652B404FF6FF552B408D8958
:100E00002B43CD892B4383800483CD888586028440
:100E100070BD70B5002400220023058C4FF6EF76DC
:100E200035400584028C8388048B48F6FF752C407E
:100E30004FF6FF452C400D884FF6FF7606EA052554
:100E40002C434FF6DF752A400D8906EA05152A4323
:100E50004D8806EA05152A43444DA84202D0494D63
:100E6000A8421DD14FF67F752A404D894FF6FF7677
:100E700006EA05152A434FF6BF752A408D8806EA13
:100E800005152A434FF6FF352B404FF2FF752B40D7
:100E90008D8906EA85052B43CD8906EA85052B4316
:100EA00083800483CD880587028470BD70B50024DB
:100EB00000220023058C4FF6FF6635400584028C26
:100EC0008388848B4FF68F752C404FF6FC752C4031
:100ED0000D882C434FF6FF552A400D894FF6FF76BB
:100EE00006EA05252A434D8806EA05252A431F4DB3
:100EF000A84202D0234DA8421DD14FF2FF752A40CF
:100F00004D894FF6FF7606EA05252A434FF6FF3551
:100F10002A408D8806EA05252A434EF6FF752B40A8
:100F20004DF6FF752B408D8906EA05152B43CD89BB
:100F300006EA05152B4383808483CD888587028448
:100F400070BD70B5002200230024058C4EF6FF769C
:100F500035400584038C8488828B48F6FF752A40CF
:100F60004FF6FF452A400D8820E00000002C01408C
:100F70000004004000080040000C00400010004049
:100F80000014004000340140004C0140005001407A
:100F90000054014000180040001C004000200040A8
:100FA0000040014000440140004801404FF6FF76F8
:100FB00006EA05252A434DF6FF752B400D8906EA02
:100FC00005352B434D8806EA05352B43FA4DA842DB
:100FD00002D0FA4DA84208D14BF6FF752C408D89FE
:100FE0004FF6FF7606EA85152C4384808283CD88F0
:100FF000A0F84050038470BD828B4FF2FF331A403B
:101000008283828B4FF6FF7303EA01231A438283A4
:101010007047F0B50C461546002200210026078CCB
:101020004EF6FF7C07EA0C070784828B018C4FF693
:10103000FF7707EA043640F6FF473A404FF6FF775E
:1010400007EA05273A434FF6FF7707EA03373A43A3
:10105000D94FB8420ED0D94FB8420BD0B0F1804F23
:1010600008D0D74FB84205D0D64FB84202D0D64F9D
:10107000B84206D14DF6FF77394046F480573943E0
:1010800005E047F6FF57394044F4805739438283DF
:101090000184F0BD828B4FF6F3731A408283828BFA
:1010A0000A4382837047F0B50C46154600220021A2
:1010B0000026078C4FF6FF6C07EA0C070784828B2B
:1010C000018C4FF6FF7707EA04264FF60C773A407B
:1010D0004FF6FF7707EA03172F433A43B64FB8425C
:1010E0000ED0B64FB8420BD0B0F1804F08D0B44FFD
:1010F000B84205D0B34FB84202D0B34FB84206D180
:101100004FF6FF57394046F48077394305E04FF2F8
:10111000FF57394044F48077394382830184F0BD1E
:10112000028B4FF2FF331A400283028B4FF6FF739C
:1011300003EA01231A4302837047F0B50C461546B3
:10114000002200210026078C4FF6EF7C07EA0C07EF
:101150000784028B018C4FF6FF7707EA041640F6EE
:10116000FF473A404FF6FF7707EA03373A434FF617
:10117000FF7707EA05273A438F4FB8420ED08F4FCB
:10118000B8420BD0B0F1804F08D08D4FB84205D097
:101190008C4FB84202D08C4FB84206D14FF6DF7761
:1011A000394046F01007394305E04FF65F77394084
:1011B00044F01007394302830184F0BD028B4FF6DF
:1011C000F3731A400283028B0A4302837047F0B51F
:1011D0000C46154600220021068C4FF6FE773E4055
:1011E0000684028B018C4FF60C7632407E1C06EA98
:1011F00003162E433243704EB0420ED06F4EB042B3
:101200000BD0B0F1804F08D06D4EB04205D06D4E7E
:10121000B04202D06C4EB04206D14FF6FD7631405E
:1012200044F00106314305E04FF6F576314044F0D5
:101230000106314302830184F0BD70B505460C46BA
:101240005D4885420ED05D4885420BD0B5F1804F98
:1012500008D05B48854205D05A48854202D05A489A
:10126000854200D100E000BF208850B92389A288C0
:1012700061882846FFF7ABFFE1882846FFF79EFF0D
:1012800025E0208804280AD12389A288618828467D
:10129000FFF753FFE1882846FFF742FF17E0208859
:1012A00008280AD12389A28861882846FFF7FBFE17
:1012B000E1882846FFF7EEFE09E02389A2886188CD
:1012C0002846FFF7A6FEE1882846FFF795FE70BD89
:1012D0002DE9F04105460C4600260127608808B933
:1012E000022600E00026A088012801D1022700E0A4
:1012F00001272088A0B92389A28861882846FFF7A2
:1013000066FFE1882846FFF759FF23893A463146B0
:101310002846FFF712FFE1882846FFF701FF13E098
:101320002389A28861882846FFF707FFE1882846BD
:10133000FFF7F6FE23893A4631462846FFF747FF76
:10134000E1882846FFF73AFFBDE8F0810A884B881C
:101350001A438B881A43CB881A430B891A434B894B
:101360001A438B891A43A0F8442070474FF6FF7147
:10137000818000210180C18041800172704700217D
:10138000018041808180C180018141818181C18151
:101390007047002101804180012181800021C180AE
:1013A000018170470021018041808180C1800181DD
:1013B0004181818170470000002C014000340140D0
:1013C0000004004000080040000C004021B10288E9
:1013D00042F00102028004E002884FF6FE731A40D8
:1013E0000280704731B1B0F8442042F40042A0F8C6
:1013F000442005E0B0F84420C2F30E02A0F84420D7
:1014000070471AB183890B43838102E083898B4340
:10141000838170478182704741EA0203A0F8483017
:1014200070471AB183890B43838102E083898B4320
:101430008381704701894FF6F8721140018170472E
:101440000A46002101894FF68F731940114301812B
:10145000704730B504460D4629462046FFF7F0FF99
:10146000208940F00700208130BD2DE9F04104467D
:101470000D4616461F46602D06D13B4601223146D9
:101480002046FFF75AFE05E03B4601223146204642
:10149000FFF79DFE29462046FFF7D2FF208940F046
:1014A00007002081BDE8F08130B50C46002101899C
:1014B000C9B24FF6FF7505EA0325154325432943B5
:1014C000018130BD2DE9F04105460E46174698468C
:1014D000002443463A4631462846FFF7E5FF2C896B
:1014E0004FF6F870044044F007044FF68F70044044
:1014F00044F070042C81BDE8F081F0B504460D463F
:1015000016461F463B46324629462046FFF7CCFF8B
:10151000208940F480402081F0BD0185828270479F
:101520000A46002101884FF68F731940114301804C
:101530007047F0B50C4615461E46002100220023D8
:101540000189028B038C4FF6F877394021434FF61F
:10155000FC473A4040F201173A434FF6DD773B40F3
:101560004FF6FF7707EA06172F433B4301810283BB
:101570000384F0BD0A460021018B4FF68F7319409A
:101580001143018370470A460021018B48F6FF731F
:1015900019404FF6FF7303EA022319430183704792
:1015A0000A460021818B4FF68F73194011438183C6
:1015B00070470A460021818B48F6FF7319404FF6A9
:1015C000FF7303EA022319438183704721B1028824
:1015D00042F08002028004E002884FF67F731A40D6
:1015E0000280704721B1828842F00402828004E0C8
:1015F00082884FF6FB731A408280704721B182883F
:1016000042F00802828004E082884FF6F7731A40A5
:101610008280704721B1828842F00102828004E01A
:1016200082884FF6FE731A40828070470A46002176
:10163000018B4FF6F77319401143018370470A4637
:101640000021018B4FF2FF7319404FF6FF7303EA3D
:1016500002231943018370470A460021818B4FF60C
:10166000F77319401143818370470A460021818B2B
:101670004FF2FF7319404FF6FF7303EA0223194339
:10168000818370470A460021018B4FF6FB73194096
:101690001143018370470A460021018B4FF6FF3347
:1016A00019404FF6FF7303EA022319430183704781
:1016B0000A460021818B4FF6FB7319401143818349
:1016C00070470A460021818B4FF6FF3319404FF6D1
:1016D000FF7303EA02231943818370470A460021FE
:1016E000018B4FF67F7319401143018370470A46FF
:1016F0000021018BC1F30E014FF6FF7303EA0223B1
:101700001943018370470A460021818B4FF67F738E
:1017100019401143818370470A460021818BC1F330
:101720000E014FF6FF7303EA0223194381837047CA
:101730000A460021018C4FF6FD73194011430184C4
:1017400070470A460021018C4FF6F7731940114388
:10175000018470470A460021018C4FF6DF7319405F
:101760004FF6FF7303EA02131943018470470A46D8
:101770000021018C4FF67F7319404FF6FF7303EA87
:1017800002131943018470470A460021018C4FF669
:10179000FF5319404FF6FF7303EA022319430184F4
:1017A00070470A460021018C4FF2FF7319404FF633
:1017B000FF7303EA02231943018470470A4600219C
:1017C000018C4DF6FF7319404FF6FF7303EA0233A5
:1017D00019430184704730B5002301248C40A3B223
:1017E000048C9C430484048C02FA01F5ADB22C43B2
:1017F000048430BD30B5002304248C40A3B2048C93
:101800009C430484048C02FA01F5ADB22C43048499
:1018100030BD70B50346002000241846183001255D
:101820008D40ACB21D8CA5431D8409B1082909D196
:1018300000EB6100056825F070050560056815433B
:1018400005600EE00D1FC5F34E052844056825F41C
:10185000E045056005684FF6FF7606EA0226354347
:10186000056070BD21B1028842F00202028004E0EE
:1018700002884FF6FD731A400280704721B102883A
:1018800042F00402028004E002884FF6FB731A4023
:101890000280704721B1828842F08002828004E099
:1018A00082884FF67F731A408280704702884FF615
:1018B000F7731A40028002880A43028070478288C8
:1018C0004FF68F731A40828082880A438280704765
:1018D00002894FF6F8731A40028102890A43028195
:1018E000704702894FF67F731A40028102890A43CA
:1018F0000281704781847047818570478186704777
:101900000187704781877047A0F8401070470288B0
:101910004FF6FF431A40028002880A430280704754
:101920000146888E70470146088F70470146888FB0
:1019300070470146B1F8400070470146888C7047F7
:101940000146088D704702460020138A0B400BB1F8
:10195000012000E000207047CA430282704730B582
:101960000246002000230024158A05EA0103958918
:1019700005EA010413B10CB1012000E0002030BDE4
:10198000CA4302827047000010B50446FB488442F7
:1019900009D101218803FFF7ABF800214FF4804003
:1019A000FFF7A6F832E0F648844209D10121480445
:1019B000FFF7ABF800214FF40030FFF7A6F825E061
:1019C000F048844209D101218804FFF79EF80021E4
:1019D0004FF48020FFF799F818E0EB48844209D1D2
:1019E0000121C804FFF791F800214FF40020FFF710
:1019F0008CF80BE0E548844208D101210805FFF787
:101A000084F800214FF48010FFF77FF810BD2DE916
:101A1000F04786B005460E460024A24600BFA14608
:101A20000027B08900B100BF2F462C8A4CF6FF700A
:101A30000440F08804432C82AC894EF6F310044035
:101A4000B08831890843718908430443AC81AC8A6A
:101A50004FF6FF400440B0890443AC8201A8FEF772
:101A600041FFC648874202D1DDF810A001E0DDF851
:101A70000CA0A88900F4004040B10AEBCA0000EBBA
:101A80000A1031684900B0FBF1F807E00AEBCA0020
:101A900000EB0A1031688900B0FBF1F86420B8FB54
:101AA000F0F004012009642101FB1089A88900F4E9
:101AB000004040B1322000EBC900B0FBF1F000F073
:101AC0000700044308E0322000EB09106421B0FB5A
:101AD000F1F000F00F0004432C8106B0BDE8F08760
:101AE0004FF41651016000218180C18001810C21D9
:101AF000418100218181704710B502460020108A83
:101B00004FF2FF0318400B884C8823438C882343F3
:101B1000CC8823431843108210BD002101804180EE
:101B20008180C180704721B1828942F40052828154
:101B300004E082894DF6FF731A4082817047F0B548
:101B40000346002400260025002040F66A17B9420B
:101B500000D100BF1846C1F3421401F01F0601274F
:101B600007FA06F5012C01D10C3004E0022C01D15A
:101B7000103000E014301AB107682F43076002E00C
:101B80000768AF430760F0BD1AB1838A0B438382B5
:101B900002E0838A8B4383827047028A4FF6F07398
:101BA0001A400282028A0A430282704782894FF2F7
:101BB000FF731A40828182890A438281704721B172
:101BC000828942F00202828104E082894FF6FD732D
:101BD0001A4082817047028A4FF6DF731A400282F0
:101BE000028A0A430282704721B1028A42F480428B
:101BF000028204E0028A4BF6FF731A4002827047A9
:101C0000C1F308028280704701468888C0F308004B
:101C10007047818941F0010181817047028BD2B206
:101C20000283028B42EA012202837047028B02F494
:101C30007F420283028B0A430283704721B1828A6A
:101C400042F02002828204E0828A4FF6DF731A405B
:101C50008282704721B1828A42F01002828204E0BF
:101C6000828A4FF6EF731A408282704721B1828ACE
:101C700042F00802828204E0828A4FF6F7731A402B
:101C80008282704721B1828942F40042828103E05E
:101C90008289C2F30E028281704721B1828A42F4A6
:101CA0000062828204E0828A4FF2FF731A408282CD
:101CB0007047828A4FF6FB731A408282828A0A43F7
:101CC0008282704721B1828A42F00202828204E05D
:101CD000828A4FF6FD731A408282704702460020C6
:101CE000B1F5007F00D100BF13880B400BB101207C
:101CF00000E00020704701F40072B2F5007F00D1CF
:101D000000BFCA430280704770B50246002400231A
:101D10000025002040F66A16B14200D100BFC1F391
:101D2000421501F01F03012606FA03F3012D02D12B
:101D30009689334006E0022D02D1168A334001E035
:101D4000968A33400C12012606FA04F416883440B1
:101D500013B10CB1012000E0002070BD10B50022CD
:101D6000002340F66A14A14200D100BF0A120124E8
:101D70009440A3B2DC43048010BD00000038014051
:101D80000044004000480040004C0040005000402B
:101D90000CB50020019000909248006840F480301B
:101DA0009049086000BF8F48006800F40030009040
:101DB0000198401C0190009818B90198B0F5A06FE7
:101DC000F1D18848006800F4003010B10120009083
:101DD00001E000200090009801285CD18248006852
:101DE00040F01000804908600846006820F00300B9
:101DF00008600846006840F00200086079484068C2
:101E0000784948600846406848600846406840F4A1
:101E1000806048600846C06A744908407149C862D9
:101E20000846C06A724908436E49C862084600689D
:101E300040F08060086000BF6A48006800F0006001
:101E40000028F9D06748406820F47C106549486054
:101E50000846406840F4E81048600846006840F0D2
:101E60008070086000BF5F48006800F000700028C4
:101E7000F9D05C48406820F003005A4948600846A1
:101E8000406840F00200486000BF5648406800F0DB
:101E90000C000828F9D10CBD10B5FFF779FF10BD73
:101EA00010B55048006840F001004E4908600846EF
:101EB0004068504908404B494860084600684E4910
:101EC0000840484908600846006820F480200860FF
:101ED0000846406820F4FE0048600846006820F08C
:101EE000A05008604FF47F0088600020C862FFF7B0
:101EF000D3FF4FF000604149086010BDF0B50021EC
:101F0000002000230024002200250026354F7F6892
:101F100007F00C0121B1042908D008294BD10BE0AE
:101F2000374FDFF8E0C0CCF800704AE0344FDFF8FC
:101F3000D4C0CCF8007044E02A4F7F6807F47010DA
:101F4000284F7F6807F48033800C0D2801D0801C57
:101F500000E0062033B92C4F4743DFF8A8C0CCF887
:101F6000007027E01F4FFF6A07F480341D4FFF6A9F
:101F700007F00F077A1C44B9214FB7FBF2F747432C
:101F8000DFF880C0CCF8007014E0164FFF6AC7F38A
:101F900003177D1C134FFF6AC7F30327BE1C184F9E
:101FA000B7FBF5F77743B7FBF2F74743DFF854C0C9
:101FB000CCF8007005E0124FDFF848C0CCF8007094
:101FC00000BF00BF074F7F68C7F30317DFF83CC0AF
:101FD0001CF807100B4F3F68CF40DFF828C0CCF843
:101FE0000070F0BD001002400020024000F0FEFF33
:101FF000140801000000FFF0FFFFF6FE08ED00E00E
:1020000000127A001400002000093D001800002092
:102010000948804709480047FEE7FEE7FEE7FEE77C
:10202000FEE7FEE7FEE7FEE7FEE7FEE704480549B8
:10203000054A064B70470000A11E00085101000828
:10204000381E0020382400203820002038200020AE
:1020500010B5002804DB0A07130E624A135406E089
:102060000A07140E604A00F00F031B1FD45410BD62
:1020700010B55E4800684FF47A71B0FBF1F4601E51
:10208000B0F1807F00D30FE0601E4FF0E021486187
:102090000F214FF0FF30FFF7DBFF00204FF0E02172
:1020A00088610720086100BF0021481EFFF7D0FFAC
:1020B00010BD10B54E4800884FF6FF71884204D01D
:1020C0004B480088401C4A4908804A4800884FF61F
:1020D000FF71884204D047480088401C4549088069
:1020E000454800884FF6FF71884204D04248008876
:1020F000401C4149088041480068401C3F49086035
:102100003F4800884FF6FF71884204D03C48008861
:10211000401C3B4908803B48008820B13948008872
:10212000401E3849088001F0E7FE01F0CBFA10BDEF
:1021300010B500214FF00060FEF7B3F84FF4A06037
:10214000FEF778F8FFF794FF00F060F800F0A0FFCA
:1021500000F016FB01F0F0F801F0B4F940F2712143
:10216000042001F085F901F089FA01F0E5F9012078
:1021700010BD10B51E4800880F2804DB00F0DBFD01
:1021800000201B4908801B480088232806DB00F03C
:10219000F0FF00F0B0FC00201649088016480088C7
:1021A00042F6E061884213DB17480078012806D127
:1021B00000201149088002201349087008E01248E5
:1021C0000078022804D100200B4908800E490870CD
:1021D00000F070F901F0F0F801F080FA01F0BDFEB6
:1021E00010BD000000E400E018ED00E01400002045
:1021F000280000202A0000202C00002030000020B1
:102200006A000020340000203D00002000B589B0A5
:1022100001210846FEF745FC01210420FEF741FCA0
:102220004FF44060ADF8040004208DF80700012051
:102230008DF8060001A9F748FEF7CAF80121C80287
:10224000FEF72FFCF448FEF791FC0121F348FEF75E
:1022500090F94FF6FF70ADF81C0040F2CF20ADF8BA
:1022600018000020ADF81E00ADF81A008DF820000F
:1022700006A9E948FEF74EFD00220121E648FFF7D6
:10228000C0F80C20ADF80C000220ADF80E000120C3
:10229000ADF810000020ADF812000520ADF81400D4
:1022A00003A9DD48FEF7C9FF1021DB48FFF754FB07
:1022B00001221021D848FFF7A4F80121D648FFF7E2
:1022C00085F91B208DF8080003208DF809000120F6
:1022D0008DF80A008DF80B0002A8FDF7B0FF012170
:1022E000CD48FFF773F8012009B000BD70B510218B
:1022F000C948FFF734FB002874D0C748FFF719FB23
:102300000546C7480068854203D9C54800682C1AAD
:1023100005E0C34800684FF6FF71081A4419C04829
:1023200005602820BF490880BF480068401CBE499E
:10233000086008460068192801D900200860BB48D9
:10234000B949096840F82140962C12D8B448006871
:10235000A04205D3B2480068001BB1490860A3E061
:10236000AF4800684FF6FF71081A2044AC49086076
:102370009AE0AF49AF4A127821F81240AD48007890
:10238000E8B9B4F5E17F0BD9B4F52A7F08D2022071
:10239000A8490870A6494C800020A74908704FE062
:1023A000B4F5617F07D940F24C40844203D200204B
:1023B000A149087070BD01209E49087040E09D4809
:1023C000007801281AD1B4F5E17F0CD9B4F52A7F41
:1023D00009D202209749087095494C8000209649FF
:1023E00008702DE064E0B4F5617F29D940F24C40DB
:1023F000844225D2002090490870DBE78D480078A0
:102400008E49097888421BDA8A480078401C89493D
:102410000870B4F5E17F08D9B4F52A7F05D202200F
:1024200008700020844908700AE0B4F5617F07D97C
:1024300040F24C40844203D200207F490870B9E743
:102440007C4800787D490978884224D102250FE034
:10245000774830F815107A480078C0EB001000EB90
:102460008000784A02EB8002A81E22F810106D1C32
:10247000724800788542EBD371480078401C70495F
:10248000087008460078062801DB0020087000204C
:102490006849087008E06748007868490978884208
:1024A00002DD00206349087010215B48FFF768FADD
:1024B00000BF7FE72DE9F04100256348007818B997
:1024C00092205E49087002E01A205C4908705C485E
:1024D00000785E49097888427DD0002404E000201D
:1024E0005B490855601C84B21E2CF8DB002489E08F
:1024F00056480078C0EB001000EB8000514901EB1A
:10250000800030F81400B0F5B47F79DD002C43DD95
:102510004E480078C0EB001000EB800001EB80011A
:10252000601E31F81000B0F58C7F1ADA4748007849
:10253000C0EB001000EB8000424901EB8001601EFF
:1025400031F81000643081B240480078C0EB0010D0
:1025500000EB80003B4A02EB8002601E22F8101064
:1025600034E03A480078C0EB001000EB80003549B9
:1025700001EB8001601C31F81000643081B23348F7
:102580000078C0EB001000EB80002E4A02EB8002C6
:10259000601C22F8101019E02C480078C0EB0010E5
:1025A00000EB8000274901EB8001601C31F810002E
:1025B000643081B225480078C0EB001000EB800049
:1025C000204A02EB8002601C22F810101F4800789D
:1025D000C0EB001001E0C6E012E000EB80001949FA
:1025E00001EB800030F81400643818490978C1EB19
:1025F000011101EB8101134A02EB810121F8140062
:10260000601C84B20D480078801EA0423FF770AF76
:1026100000244EE000080140002C0140400016005C
:10262000440000203400002040000020B4110020AD
:102630002C1200203C00002049000020390000201E
:102640003B0000208C0A0020890A00203A0000206C
:1026500094110020E11704EB5171C1F3CF06E1178B
:1026600004EB5171C910A4EBC1018FB23F4800784F
:10267000C0EB001000EB80003D4901EB800030F81A
:102680001400FA2813DD39480078C0EB001000EB85
:10269000800001EB800030F81400B0F5FA7F06DA14
:1026A0003448805D0121B940084332498855601C97
:1026B00084B231480078801EA042CBDC2F480078DD
:1026C00008BB0025002405E02A48005D284485B2A7
:1026D000601C84B2112CF7DB2648407C00F00F0010
:1026E000284485B22348407C040905F00F00A0422D
:1026F0002ED12048407C00F00F001E494874084647
:1027000002F064F824E01B48057840780544194835
:10271000807800F00F00054416488078040905F021
:102720000F00A04209D11348807800F00F00114932
:102730008870084602F04AF80AE00E48807843287C
:1027400003D00C488078532802D10A4802F0BCF923
:1027500006480078401C054908700846007806289D
:1027600001DB00200870BDE8F08100003A00002085
:102770008C0A00209411002039000020890A0020D2
:1027800000B585B001211020FEF798F9FE48FEF74C
:10279000EDF94720ADF808000020ADF80E00ADF8C7
:1027A0000A006320ADF80C0002A9F748FEF7B2FA60
:1027B00001221146F448FEF724FE00220121F248CE
:1027C000FEF71FFE0121F048FFF7C6F836208DF80E
:1027D000040002208DF8050000208DF8060001207D
:1027E0008DF8070001A8FDF72AFD0121E648FEF754
:1027F000EDFD01210420FEF754F94FF40070ADF80F
:10280000000010208DF8030003208DF802006946B7
:10281000DE48FDF7DDFD4FF40071DC48FDF787FE73
:1028200001210420FEF73DF94FF48070ADF800005F
:1028300004208DF8030003208DF802006946D34878
:10284000FDF7C6FD0020D2490870012005B000BD8B
:1028500001B50020BDF800100812BDF800100144B9
:10286000C8B29DF8021001F00F018DF802109DF81A
:1028700002100144C8B29DF8021000F00F0241EAB4
:1028800002118DF80210BDF800100912C14A117032
:10289000BDF8001051709DF8021091701146097832
:1028A00001F00101BC4A1170BA490978C1F3400135
:1028B0005170B8490978C1F380019170B549097820
:1028C000C1F3C001D170B3490978C1F3001111718E
:1028D000B0490978C1F340115171AE490978C1F38B
:1028E00080119171AB490978C909D171A949497819
:1028F00001F001011172A7494978C1F340015172F9
:10290000A4494978C1F380019172A2494978C1F381
:10291000C001D1729F494978C1F3001111739D49DB
:102920004978C1F3401151739A494978C1F3801134
:10293000917398494978C909D1739649897801F00A
:102940000101117493498978C1F34001517491498F
:102950008978C1F3800191748E498978C1F3C001EF
:10296000D1748C498978C1F300111175894989782E
:10297000C1F34011517587498978C1F38011917570
:1029800084498978C909D1750121844A117008BD2B
:1029900001B500209DF8021001F00F018DF8021022
:1029A0009DF802100907090E7A4A1170114609783C
:1029B000BDF8002041EA2231764A1170BDF80010BE
:1029C000C1F303210901517011464978BDF8002077
:1029D000C2F3031211436F4A5170BDF8001001F0A9
:1029E0000F0191701146097852781144694A927822
:1029F000114401F00F006749897841EA0011654AE6
:102A000091701146097801F00101634A1170614922
:102A10000978C1F3400151705E490978C1F3800122
:102A200091705C490978C1F3C001D17059490978A6
:102A3000C1F30011117157490978C1F34011517167
:102A400054490978C1F38011917152490978C90933
:102A5000D1715049497801F0010111724D4949780D
:102A6000C1F3400151724B494978C1F38001917221
:102A700048494978C1F3C001D17246494978C1F348
:102A80000011117343494978C1F340115173414911
:102A90004978C1F3801191733E494978C909D173CE
:102AA0003C49897801F0010111743A498978C1F3F0
:102AB0004001517437498978C1F3800191743549D7
:102AC0008978C1F3C001D17432498978C1F300110A
:102AD000117530498978C1F3401151752D498978B4
:102AE000C1F3801191752B498978C909D1750121EC
:102AF0002A4A117008BD10B529480078401C2849A1
:102B00000870084600781E2800DA10BD64202449A9
:102B1000087080212348FDF7EEFC80212148FDF755
:102B2000EAFC78B320480078401C1F490870002058
:102B30001E4908701C4800781E2877DD00201A49BD
:102B4000087001201A490870084600781949097868
:102B5000884200D1D9E7012017490870154908704B
:102B60004FF65972092100F0EFFD4FF65972092115
:102B7000012000F0E9FD4FF659720921012000F013
:102B8000E3FD1BE01FE000000010004000080140D2
:102B9000490000204B000020BC1300205000002002
:102BA000510000200010014052000020530000207E
:102BB0005400002055000020480000208021FE48DD
:102BC000FDF7B5FC32E0FD480078401CFB49087079
:102BD0000020FB490870F94800781E2826DD0020F7
:102BE000F6490870F749087008460078F6490978F0
:102BF000884200D189E70020F4490870F249087042
:102C00004FF64E720921012000F09EFD4FF64E72E4
:102C10000921012000F098FD4FF64E720921012094
:102C200000F092FD8021E448FDF77FFC00BF6CE7D7
:102C300010B50121E648FEF792FE012879D1012165
:102C4000E348FEF79DFEE34800780A2809DB4FF4CD
:102C50000070E1490860DF480078401EDD490870D7
:102C600010BDDC48007809280DDCDA48007850B146
:102C70004FF40070D849091D0860D6480078401EFE
:102C8000D4490870ECE7D5480078002851DDD148D8
:102C9000007800284DD1D148007801280CD1292096
:102CA000CC4908704FF40070CB490860CB480078DD
:102CB000401CCA4908703CE0C84800781B2816DA56
:102CC000C6480078801EC649085C18B11B20C1495F
:102CD000087002E01120BF4908704FF40070BE492F
:102CE0000860BE480078401CBC49087021E0BB4821
:102CF00000781B280DD10020B64908704FF40070F1
:102D0000B549091D0860B5480078401CB3490870F2
:102D10000FE00020B14908704FF40070AE49091D62
:102D200008600020AB49087000220121A848FEF786
:102D300068FB00BF94E710B5AA48007868B1AA48BC
:102D40000078401CA849087008460078052803DB75
:102D500000200870A349087010BD0020A249087027
:102D6000A248008800B1F7E7012000F061FE0446A8
:102D7000207840B12078102805DA608822789C4BB2
:102D800053F82210884700BFE6E700BF704738B508
:102D9000044600200090ADF8004004208DF80200A9
:102DA0000098FFF755FD01208C490870012211465B
:102DB0008748FEF726FB8F48007848B18D48007899
:102DC000401E8C49087022460121084600F0BCFCD8
:102DD00038BD38B5044600200090ADF8004005200D
:102DE0008DF802000098FFF733FD01207B49087041
:102DF000012211467648FEF704FB7E48007848B170
:102E00007C480078401E7B49087022460221012040
:102E100000F09AFC38BD38B5044600200090ADF8AB
:102E2000004006208DF802000098FFF711FD0120F8
:102E30006A490870012211466548FEF7E2FA38BD7A
:102E400038B5044600200090ADF8004007208DF80A
:102E500002000098FFF7FCFC012060490870012285
:102E600011465B48FEF7CDFA38BD38B50446002060
:102E70000090ADF8004002208DF802000098FFF7A6
:102E8000E7FC012055490870012211465048FEF721
:102E9000B8FA38BD38B5044600200090ADF80040BF
:102EA00003208DF802000098FFF7D2FC01204B4967
:102EB0000870012211464648FEF7A3FA38BD38B51E
:102EC000044600200090ADF8004001208DF802007B
:102ED0000098FFF7BDFC012040490870012211460F
:102EE0003B48FEF78EFA38BD38B504460020009006
:102EF000ADF8004008208DF802000098FFF7A8FC0C
:102F0000012036490870012211463148FEF779FA4E
:102F100038BD38B5044600200090ADF800400920C7
:102F20008DF802000098FFF793FC01202B490870F0
:102F3000012211462648FEF764FA38BD38B504462A
:102F400000200090ADF800400D208DF802000098A0
:102F5000FFF77EFC012021490870012211461C4820
:102F6000FEF74FFA38BD38B5044600200090ADF8A2
:102F700000400E208DF802000098FFF769FC012048
:102F800016490870012211461148FEF73AFA38BD79
:102F900038B5044600200090ADF800400F208DF8B1
:102FA00002000098FFF754FC01200C490870012230
:102FB0001146074820E00000000C014053000020AB
:102FC000520000205400002055000020480000203E
:102FD0000010004056000020100801404F00002063
:102FE000BC130020500000205700002034000020B7
:102FF000704C000849000020FEF703FA38BD38B5D0
:10300000044600200090ADF800400A208DF8020030
:103010000098FFF71DFC01201A4908700122114693
:103020001948FEF7EEF938BD38B504460020009087
:10303000ADF80040154800788DF802000098FFF7C1
:10304000A7FC01200F490870012211460E48FEF727
:10305000D8F938BD38B5044600200090ADF80040DE
:103060000A48007840F008008DF802000098FFF749
:103070008FFC012003490870012211460248FEF727
:10308000C0F938BD4F000020001000404A00002069
:1030900000B587B001210846FDF703FD012104209A
:1030A000FDF7FFFC01210420FDF7FBFC18208DF843
:1030B0001B0003208DF81A000420ADF8180006A9A3
:1030C0009248FDF785F904208DF81B000820ADF823
:1030D000180006A98D48FDF77BF901214804FDF78A
:1030E000EDFC8B48FEF750FC4FF4E13001900020DE
:1030F000ADF80800ADF80A00ADF80C000C20ADF8F2
:103100000E000020ADF8100001A98148FEF77FFCF9
:1031100001217F48FEF707FD40F225517C48FEF76C
:103120001DFE40F227717A48FEF718FE012240F298
:1031300025517748FEF703FD26208DF81400032063
:103140008DF8150000208DF8160001208DF817006D
:1031500005A8FDF774F800206E4908606E49086004
:103160006E4908606E4908606E490870012007B01A
:1031700000BD10B56B48007800BB6848006868491E
:10318000096888421AD0FF206649087064480468BC
:103190000068401C6249086008460068B0F5806F0E
:1031A00001D3002008606048015D5948FEF728FD02
:1031B000012240F227715648FEF7C1FC55480068CD
:1031C00055490968884243D03CE05848524909684B
:1031D000405C242806D10020554908602420554928
:1031E000087018E051484C490968405C23280AD10E
:1031F00050494F4A12688854084600F0ACFF00203E
:103200004B49086007E0494843490968405C49491F
:10321000474A1268885446480068401C4449086080
:1032200008460068642801D3002008603A48006816
:10323000401C3949086008460068B0F5806F01D32A
:103240000020086033480068334909688842BCD1CF
:1032500010BD10B513E00278334B304C24681A557A
:103260002E4A1268521C2D4B1A601A461268B2F58B
:10327000806F01D300221A60401C4A1E91B20029BF
:10328000E9DC10BD10B540F225512148FEF73CFDA8
:1032900090B11F48FEF7B8FC24491E4A12688854B2
:1032A0001C480068401C1B49086008460068B0F5CF
:1032B000806F01D30020086040F227711448FEF7A8
:1032C00023FD08B31648006814490968884212D0E3
:1032D000134804680068401C1149086008460068EB
:1032E000B0F5806F01D3002008600F48015D0848E9
:1032F000FEF786FC08E000200A490870002240F230
:1033000027710348FEF71BFC10BD000000080140B8
:1033100000440040580000205C00002060000020B5
:103320006400002068000020DA170020DA13002073
:1033300070000020DA1B002008B501210820FDF7ED
:10334000B0FB10208DF8030002208DF802008003EE
:10335000ADF8000069464148FDF73AF84FF40041E6
:103360003E48FDF7E4F801210820FDF79AFB102004
:103370008DF8030002208DF802004003ADF8000034
:1033800069463648FDF724F84FF480413348FDF78D
:10339000CEF810208DF8030002208DF80200802066
:1033A000ADF8000069462D48FDF712F800202C49C1
:1033B00008704870012008BD10B52A4800682A49E5
:1033C000096888420FD92748006800F5FA70264935
:1033D00008602648007818B901202449087002E0E6
:1033E0000020224908701E48407850B1012802D0C0
:1033F000022814D10BE04FF400411848FDF795F86E
:103400000DE04FF400411548FDF791F807E017482B
:1034100002784FF400411148FDF78BF800BF00BF60
:103420000F48007850B1012802D0022814D10BE0D7
:103430004FF480410948FDF778F80DE04FF48041E2
:103440000648FDF774F807E0084802784FF4804119
:103450000248FDF76EF800BF00BF10BD000C014030
:103460007400002030000020780000207C00002044
:1034700045F25552084B1A601A46506091604AF660
:10348000AA221A604CF6CC421A6070474AF6AA206B
:1034900001490860704700000030004010B500246A
:1034A00004212248FDF743F800BF02E0FFF7EEFFDA
:1034B000641C1F488442F9D304211C48FDF735F8E9
:1034C000012010BD08B501213020FDF7EAFA1020D7
:1034D0008DF8030002208DF802000420ADF80000F2
:1034E00069461248FCF774FF04211048FDF71DF8E7
:1034F000FFF7D4FF10208DF8030002208DF80200A2
:10350000ADF8000069460B48FCF762FF012008BDDA
:1035100010B5044624B102210648FDF706F803E081
:1035200002210448FDF703F810BD0000001401401B
:1035300020A107000010014008B501210820FDF777
:10354000B0FA01211020FDF7ACFA01211020FDF79F
:10355000A8FA01210420FDF7A4FA10208DF8030039
:1035600002208DF80200ADF8000069463F48FCF7E4
:103570002FFF02213D48FCF7D8FF28208DF80300DB
:1035800002208DF802001020ADF80000694638488E
:10359000FCF71EFF48208DF8030002208DF8020082
:1035A0000120ADF8000069463148FCF711FF012108
:1035B0002F48FCF7BAFF10208DF8030002208DF889
:1035C00002000003ADF8000069462848FCF700FF40
:1035D0004FF400512548FCF7A8FF10208DF8030098
:1035E00002208DF80200C002ADF8000069462148B3
:1035F000FCF7EEFE4FF480511E48FCF798FF08BD23
:1036000010B510211A48FCF776FF1B4908700846D0
:10361000007810BD10B5044624B102211348FCF710
:1036200084FF03E002211148FCF781FF10BD10B5B3
:1036300004462CB14FF400510C48FCF776FF04E02F
:103640004FF400510948FCF772FF10BD10B5044655
:103650002CB14FF480510748FCF767FF04E04FF4AA
:1036600080510448FCF763FF10BD0000000C0140CE
:1036700000100140000801407D00002008B5012134
:103680001020FDF70EFA48208DF8030002208DF877
:1036900002004020ADF8000069462748FCF798FE7C
:1036A00048208DF8030002208DF802008020ADF83C
:1036B000000069462048FCF78BFEFF201F49087078
:1036C000012008BD1E4800884FF6FF71884204D0D3
:1036D0001B480088401C1A490880704710B5002418
:1036E00040211548FCF707FF04468CB115480078C7
:1036F000401C1449087008460078C8281BDD0020CB
:103700000870FF200D49087000200D49088012E064
:1037100000200C4908700A48008864280BDD07481F
:103720000078012804D0FFF7B9FE0120FFF7F0FE72
:1037300001200249087010BD001001407E000020E9
:10374000800000207F000020F8B50B468DF8003087
:10375000ADF8022000EB4006C6EB8016E64F17F8E6
:10376000166006F07F0100EB4006C6EB801617F8E6
:10377000166006F0800500EB4006C6EB801607EBEE
:103780004606767806F07F0495B900EB4006C6EB56
:10379000801607EB4606B61C06EB8106009F3760D5
:1037A0004E1CF1B21E2900D30021A14200D10125F7
:1037B0000DB141F0800100EB4006C6EB8016CE4F04
:1037C00007F8161000EB4006C6EB801607EB46061E
:1037D0007470F8BD2DE9F8410C4615468DF800408F
:1037E000ADF8025000EB4007C7EB8017DFF808C3C5
:1037F0001CF8177007F07F0100EB4007C7EB80173C
:103800001CF8177007F0800600EB4007C7EB801725
:103810000CEB47077F7807F07F03EEBB1A4624E0E6
:1038200000EB4007C7EB8017DFF8CCC20CEB470773
:10383000BF1C17F822709DF800C0674510D1BDF875
:1038400002C000EB4007C7EB8017DFF8AC8208EB43
:103850004707BF1C07EB8207A7F802C0BDE8F88145
:10386000571CFAB21E2A00D300228A42D8D100EB9C
:103870004007C7EB8017DFF880C20CEB4707BF1C7F
:1038800007EB8107DDF800C0C7F800C04F1CF9B294
:103890001E2900D3002100E002E0994200D1012658
:1038A0000EB141F0800100EB4007C7EB8017DFF855
:1038B00048C20CF8171000EB4007C7EB80170CEB61
:1038C00047077B7000BFC9E7F8B50C4615468DF871
:1038D0000040ADF8025000EB4007C7EB8017DFF85F
:1038E00018C21CF8177007F07F0100EB4007C7EB08
:1038F00080171CF8177007F0800600EB4007C7EB35
:1039000080170CEB47077F7807F07F037EBB1A46D2
:1039100014E000EB4007C7EB8017DFF8DCC10CEBCD
:103920004707BF1C17F822709DF800C0674500D1FB
:10393000F8BD571CFAB21E2A00D300228A42E8D1F1
:1039400000EB4007C7EB8017DFF8ACC10CEB470773
:10395000BF1C07EB8107DDF800C0C7F800C04F1C93
:10396000F9B21E2900D30021994200D101260EB1DF
:1039700041F0800100EB4007C7EB8017DFF878C10A
:103980000CF8171000EB4007C7EB80170CEB47074C
:103990007B7000BFCCE7F8B50B4614468DF80030BD
:1039A000ADF8024000EB4006C6EB8016524F17F808
:1039B000166006F07F0100EB4006C6EB801617F894
:1039C000166006F0800500EB4006C6EB801607EB9C
:1039D0004606767806F07F0225B109B91D2101E07F
:1039E0004E1EF1B20AB91D2201E0561EF2B200EBE2
:1039F0004006C6EB8016404F07EB4606B61C06EBAA
:103A00008206009F3760914200D101250DB141F03F
:103A1000800100EB4006C6EB8016374F07F8161002
:103A200000EB4006C6EB801607EB46067270F8BD49
:103A300030B501460020314D287001EB4100C0EB4C
:103A400081102D4D15F8100000F07F0301EB4100AF
:103A5000C0EB811005EB4000407800F07F0201EBE5
:103A60004100C0EB811005EB4000407800F080047D
:103A70009CB901EB4100C0EB811005EB4000801CBC
:103A800000EB82051D482D680560501CC2B21E2A3D
:103A900000D30022934200D101240CB142F08002F5
:103AA00001EB4100C0EB8110134D05F8103001EB24
:103AB0004100C0EB811005EB400042700F4830BD63
:103AC000002100EB4002C2EB80120B4B03F81210F6
:103AD000802100EB4002C2EB801203EB42025170E6
:103AE000704710B5002404E02046FFF7E9FF601C92
:103AF000C4B2032CF8DB10BD3E1C00208200002065
:103B0000002106E00A2100BF0A1EA1F1010399B2BB
:103B1000FAD1021EA0F1010398B2F3D1704738B573
:103B20000446012C03D110208DF8030002E0482048
:103B30008DF8030002208DF802000120ADF800008E
:103B40006946EB48FCF744FC38BD10B50120FFF78F
:103B5000E6FF0121E648FCF7E8FC10BD10B50120A6
:103B6000FFF7DDFF0121E248FCF7E1FC10BD10B5D5
:103B70002021E048FCF7D9FC10BD10B52021DD481C
:103B8000FCF7D5FC10BD08B501211820FCF789FF12
:103B900010208DF8030002208DF802000120ADF8FE
:103BA00000006946D248FCF713FC10208DF8030092
:103BB00002208DF802002020ADF800006946CD48B3
:103BC000FCF706FC012008BD10B5FFF7DCFFFFF78E
:103BD000CEFFFFF7BAFF10BD10B50120FFF79FFF22
:103BE000FFF7C5FF0A20FFF78BFFFFF7AEFF1E2090
:103BF000FFF786FFFFF7B2FF1E20FFF781FFFFF7F9
:103C0000BCFF10BD10B50120FFF789FFFFF7A6FF2D
:103C10000A20FFF775FFFFF7AAFF0A20FFF770FFE2
:103C2000FFF793FF0A20FFF76BFF10BD10B50120CF
:103C3000FFF775FFFFF789FF1E20FFF761FFFFF712
:103C400096FF1E20FFF75CFF10BD10B50120FFF7A7
:103C500066FFFFF792FF0A20FFF752FFFFF77EFF94
:103C60000A20FFF74DFFFFF782FF0A20FFF748FF0A
:103C7000FFF783FF0A20FFF743FF10BD10B50120B7
:103C8000FFF74DFFFFF779FF0A20FFF739FFFFF736
:103C90005CFF0A20FFF734FFFFF769FF0A20FFF7F8
:103CA0002FFFFFF76AFF0A20FFF72AFF10BD10B5AC
:103CB0000120FFF734FFFFF748FF0A20FFF720FF3E
:103CC0000020FFF72CFF0A20FFF71AFFFFF74FFF36
:103CD0000A20FFF715FF01218548FCF70CFC08B10D
:103CE000002400E00124FFF748FF0A20FFF708FF47
:103CF000204610BD70B505460120FFF710FF0824CF
:103D000019E0601E45FA00F000F0010010B1FFF765
:103D10001CFF01E0FFF722FF0A20FFF7F1FEFFF78B
:103D200026FF0A20FFF7ECFEFFF727FF0A20FFF728
:103D3000E7FE601EC4B2012CE3DA70BD70B5054623
:103D4000002600240020FFF7EAFE00BF14E0FFF782
:103D500014FF0A20FFF7D4FEFFF709FF6006040EE8
:103D600001216348FCF7C7FB08B144F001040A20B5
:103D7000FFF7C6FE701CC6B2072EE8DD012D02D18A
:103D8000FFF77CFF01E0FFF760FF204670BD70B5D4
:103D90000024002514E06006040EFFF7E8FE0A2068
:103DA000FFF7AEFE01215248FCF7A5FB08B1601CED
:103DB000C4B2FFF7E2FE0A20FFF7A2FE681CC5B2FC
:103DC000082DE8DB204670BD70B504460D46FFF7B0
:103DD00003FFC020FFF78EFFFFF769FF0646FC20B8
:103DE000FFF788FFFFF763FFF320FFF783FFFFF77D
:103DF0005EFF3B20FFF77EFFFFF759FF2012FFF722
:103E000079FFFFF754FFE0B2FFF774FFFFF74FFFB2
:103E10002812FFF76FFFFFF74AFFE8B2FFF76AFFCC
:103E2000FFF745FFFFF7EEFE70BD2DE9F0410746B5
:103E30000C461546FFF7D0FEC020FFF75BFFFFF7EB
:103E400036FF064608E02878FFF754FFFFF72FFFFC
:103E50000646601E84B26D1C002CF4D1FFF7D2FE22
:103E6000BDE8F0812DE9F04106460C461746FFF704
:103E7000B3FEC020FFF73EFFFFF719FF0546FC2009
:103E8000FFF738FFFFF713FF0546F320FFF732FF78
:103E9000FFF70DFF05463720FFF72CFFFFF707FF61
:103EA00005463820FFF726FFFFF701FF05460720EC
:103EB000FFF720FFFFF7FBFE0546FFF7A3FEFFF726
:103EC0008BFEC120FFF716FFFFF7F1FE054600202D
:103ED000FFF734FF2070641CFFF7B7FE0020FFF7E8
:103EE0002DFF2070FFF7CAFEFFF78CFEBDE8F081C2
:103EF000000C0140001001404B4800884FF6FF7154
:103F0000884204D048480088401C474908807047D0
:103F100070B505460C46FFF75FFE012C02D1C020AC
:103F2000FFF7E8FE4148007808B9002070BD0AE0BC
:103F30006D1C2878FFF7DEFE3C48007808B90020A9
:103F4000F4E7601E84B2002CF2DCFFF75BFE012078
:103F5000ECE710B5FFF738FE10BD10B53448007817
:103F600006285ED2DFE800F00310233D565C0020F7
:103F70002D4908802F490870FFF74CFB2C4800782A
:103F8000401C2B4908704DE027480088C82800DAFB
:103F900048E00120FFF73EFBFFF7DBFF002022494E
:103FA000088023480078401C214908703AE01E48E8
:103FB0000088B0F5FA6F00DA34E01F4A40F242316F
:103FC000C020FFF732FF1B480078401C19490870D9
:103FD00000201549088016480078401C14490870D4
:103FE00020E011480088B0F57A7F00DA1AE000205E
:103FF000FFF71DFBFFF704FB28B10E480078401CBB
:104000000C49087002E000200A49087000200649A7
:10401000088007E006480078401C0549087001E068
:1040200000E000BF00BF10BD8A0000208600002015
:1040300089000020640A00201A070020FEF778F8A3
:10404000FFF74FFD0020FE494870FE490870FE480A
:104050000068FE4908600020FD49087036E0FD4810
:104060000078002805DDFB480078401EF9490870FB
:1040700004E0FF20F7490870FFF708FAF1480078DC
:10408000002817DDF0480068F049096888420DD91A
:10409000EE4800684CF25031884207D9FFF7FEF92C
:1040A0000020E8490870E649487008700120E4499A
:1040B000487009E0E44800684CF250310844E34994
:1040C00008600020DE494870FEF753F8C7E7F0B5F6
:1040D00085B005460E4614461422DFA1684600F05E
:1040E00057FD05B114B9002005B0F0BD00270FE061
:1040F0002878694601EB2010007804F8010B287835
:1041000000F00F001DF8000004F8010B6D1C7F1C6F
:10411000B742EDD3202020707000E5E7024600236F
:10412000302A05DB392A03DCA2F13000C3B202E0F9
:10413000A2F13700C3B21807030E302906DB392974
:1041400004DCA1F130001843C0B27047A1F1370080
:104150001843C0B2F9E738B50446002000906078F3
:10416000082815DA6078C14908702079E17800EBF9
:10417000012082B20E210120FFF7E6FAA0796179D1
:1041800000EB012082B20F210120FFF7DDFA38BDDC
:104190006078442872D00ADCA0F130000A281BD2D3
:1041A000DFE800F01A1B344774AAC8FCFAF9522859
:1041B0007ED008DC45287CD046287BD047287AD0A2
:1041C000482809D1CFE2532876D0572875D05928EE
:1041D00074D05A28F5D1C5E2F5E2E07857280AD123
:1041E000002098490870984800684AF6C871084449
:1041F0009649086009E001209249087092480068D9
:104200004AF6C871084491490860DCE2E078302839
:1042100002D1FFF743F905E0E078312802D101200F
:10422000FFF776F9002087490870854948700870C3
:10423000C9E2E078302803D102208149087024E0E7
:10424000E07831281BD101207D490870884800782A
:10425000D8B90120864908704FF659720821FFF736
:1042600073FA4FF6597208210120FFF76DFA4FF6E5
:10427000597208210120FFF767FA06E097E1E0781C
:10428000322802D100206E4908709CE20020FFF71E
:10429000DDF92179E078FFF741FF8DF80000A17981
:1042A0006079FFF73BFF8DF801007248007806E067
:1042B00088E2AAE1CCE19FE026E2EBE054E230B1F3
:1042C0004FF6597209210120FFF73EFA05E04FF63B
:1042D0004E7209210120FFF737FA9DF801009DF881
:1042E000001000EB012082B201210846FFF72CFAF2
:1042F00002206149087066E20020FFF7A7F92179E2
:10430000E078FFF70BFF8DF80000A1796079FFF7E7
:1043100005FF8DF801009DF801009DF8001000EBED
:10432000012082B202210120FFF70EFA0220524939
:10433000087048E20120FFF789F92179E078FFF75A
:10434000EDFE8DF80000A1796079FFF7E7FE8DF8AA
:1043500001009DF801009DF8001000EB012082B2E1
:1043600003210120FFF7F0F99DF801009DF80010EE
:1043700000EB012082B203210120FFF7E5F99DF84F
:1043800001009DF8001000EB012082B20321012002
:10439000FFF7DAF917E2D9E0AAE0FFE72179E07840
:1043A000FFF7BCFE8DF80000A1796079FFF7B6FE3B
:1043B0008DF801009DF801009DF8001000EB012030
:1043C00082B204210120FFF7BFF99DF801009DF89A
:1043D000001000EB012082B204210120FFF7B4F9A4
:1043E0009DF801009DF8001000EB012082B204212D
:1043F0000120FFF7A9F9E6E12179E078FFF78EFEC9
:104400008DF80000A1796079FFF788FE8DF8010032
:104410009DF801009DF8001000EB012082B20A21F6
:104420000120FFF791F99DF801009DF8001000EBC5
:10443000012082B20A210120FFF786F91EE0000068
:1044400074000020880A002030000020840A002028
:1044500089000020680A0020303132333435363785
:104460003839414243444546000000004A000020DC
:10447000890A002048000020490000209DF8010022
:104480009DF8001000EB012082B20A210120FFF705
:104490005BF998E12179E078FFF740FE8DF80000A4
:1044A000A1796079FFF73AFE8DF801009DF80100CF
:1044B0009DF8001000EB012082B20B210120FFF7D4
:1044C00043F99DF801009DF8001000EB012082B235
:1044D0000B210120FFF738F99DF801009DF800102D
:1044E00000EB012082B20B210120FFF72DF96AE1D8
:1044F0002179E078FFF712FE8DF80000A17960794C
:10450000FFF70CFE8DF801009DF801009DF80010EA
:1045100000EB012082B205210120FFF715F99DF87B
:1045200001009DF8001000EB012082B2052101205E
:10453000FFF70AF99DF801009DF8001000EB01203B
:1045400082B205210120FFF7FFF83CE12179E078F4
:10455000FFF7E4FD8DF80000A1796079FFF7DEFD3B
:104560008DF801009DF801009DF8001000EB01207E
:1045700082B206210120FFF7E7F89DF801009DF8BF
:10458000001000EB012082B206210120FFF7DCF8C9
:104590009DF801009DF8001000EB012082B2062179
:1045A0000120FFF7D1F80020FB4908700BE12179C9
:1045B000E078FFF7B3FD8DF80000A1796079FFF78F
:1045C000ADFD8DF801009DF801009DF8001000EB95
:1045D000012082B207210120FFF7B6F89DF8010003
:1045E0009DF8001000EB012082B207210120FFF7A7
:1045F000ABF89DF801009DF8001000EB012082B29D
:1046000007210120FFF7A0F8DDE0E079592803D168
:104610000120E249087002E00020E0490870E079DA
:1046200000F57F4082B208210120FFF78DF8E07984
:1046300000F57F4082B208210120FFF785F8E0797C
:1046400000F57F4082B208210120FFF77DF8BAE033
:10465000E079312829D1D248007850B9002142F2BE
:104660000C30FFF7B1FB4FF4805142F20D30FFF7F1
:10467000ABFB0120CA490870E07900F57F4082B2A7
:1046800009210120FFF760F8E07900F57F4082B250
:1046900009210120FFF758F8E07900F57F4082B248
:1046A00009210120FFF750F82DE0E07930282AD1C8
:1046B000BB48007801280BD14FF4207142F20C3036
:1046C000FFF782FB4FF4805142F20D30FFF77CFB85
:1046D0000020B3490870E07900F57F4082B20921DB
:1046E0000120FFF731F8E07900F57F4082B209211F
:1046F0000120FFF729F8E07900F57F4082B2092117
:104700000120FFF721F85EE02179E078FFF706FD50
:104710008DF80000A1796079FFF700FD8DF80100A8
:104720009DF801009DF8001000EB012082B20C21E1
:104730000120FFF709F89DF801009DF8001000EB3B
:10474000012082B20C210120FEF7FEFF9DF801003E
:104750009DF8001000EB012082B20C210120FEF731
:10476000F3FF30E000BF00BF2179E078FFF7D6FC0F
:104770008DF80000A1796079FFF7D0FC8DF8010079
:104780009DF801009DF8001000EB012082B20D2180
:104790000120FEF7D9FF9DF801009DF8001000EB05
:1047A000012082B20D210120FEF7CEFF9DF801000D
:1047B0009DF8001000EB012082B20D210120FEF7D0
:1047C000C3FF00E000BF00BF00BFE0E430B589B028
:1047D00004460120714908700846007838BB002063
:1047E0007049088024208DF8040045208DF80500CC
:1047F0002C208DF806000DF1070202212046FFF75C
:1048000066FC002506E0A81C215CE81D01AA1154E5
:10481000681CC5B20F2DF6DB40208DF81A0023204E
:104820008DF81B00182101A8FEF713FD4AE1A078BE
:104830000A2805D0A0780B2802D0A0780C284BD1EC
:1048400024208DF80400A078092805DCA0783030F9
:10485000C0B28DF8050004E0A0783730C0B28DF802
:1048600005002C208DF806000DF1070202212046DC
:10487000FFF72DFC31208DF80B0023208DF80C0064
:10488000494800782178884209D1474840786178C2
:10489000884204D144488078A178884209D02078A1
:1048A0004149087060784870A078887000203A49C3
:1048B0000870A0780C280AD13748007818B9092167
:1048C00001A8FEF7C6FC012033490870FAE009216F
:1048D00001A8FEF7BEFCF5E0A0780E280FD1304805
:1048E00000780128A2D1002142F20C30FFF76CFAC7
:1048F0004FF4805142F20D30FFF766FAE2E0A07803
:104900000F280FD12648007801288FD14FF420714D
:1049100042F20C30FFF758FA002142F20D30FFF757
:1049200053FACFE0A078012819D124208DF8040093
:1049300051208DF805002C208DF806000DF107029E
:1049400002212046FFF7C3FB31208DF80B00232006
:104950008DF80C00092101A8FEF77BFCB2E0A078DD
:10496000022823D124208DF804005A208DF8050058
:104970002C208DF806000DF1070202212046FFF7DA
:10498000A6FB31208DF80B0023208DF80C000921A7
:1049900001A8FEF75EFC95E03D000020890A00209A
:1049A0008A0A00206A000020CA1D0020A07803287F
:1049B00019D124208DF8040048208DF805002C2002
:1049C0008DF806000DF1070202212046FFF77FFB5C
:1049D00031208DF80B0023208DF80C00092101A84F
:1049E000FEF737FC6EE0A078042819D124208DF85A
:1049F000040059208DF805002C208DF806000DF1DB
:104A0000070202212046FFF762FB31208DF80B00E0
:104A100023208DF80C00092101A8FEF71AFC51E0B3
:104A2000A078052819D124208DF8040052208DF893
:104A300005002C208DF806000DF10702022120460A
:104A4000FFF745FB31208DF80B0023208DF80C007B
:104A5000092101A8FEF7FDFB34E0A078072831D139
:104A600024208DF8040050208DF805002C208DF8AE
:104A700006000DF1070202212046FFF728FB312036
:104A80008DF80B0023208DF80C003E48007821782B
:104A9000884209D13B4840786178884204D139483E
:104AA0008078A17888420AD02078364908706078EA
:104AB0004870A0788870092101A8FEF7CAFB002081
:104AC0003149087009B030BD10B588B004460020E7
:104AD0002D4908704FF6597208210120FEF734FE67
:104AE0004FF6597208210120FEF72EFE4FF659723B
:104AF00008210120FEF728FE207800F0F0001028A1
:104B00001CD124208DF8000041208DF801002C20BC
:104B10008DF802000DF1030202212046FFF7D7FABB
:104B200031208DF8070023208DF808000020174958
:104B3000088009216846FEF78CFB20E0207800F011
:104B4000F00030281BD124208DF8000043208DF880
:104B500001002C208DF802000DF1030202212046F5
:104B6000FFF7B5FA31208DF8070023208DF80800F3
:104B700000200649088009216846FEF76AFB08B054
:104B800010BD0000CA1D00203D0000206A0000206A
:104B900010B5203AC0F00B80B1E81850203AA0E8D8
:104BA0001850B1E81850A0E81850BFF4F5AF5FEA0C
:104BB000027C24BFB1E81850A0E8185044BF18C9BF
:104BC00018C0BDE810405FEA827C24BF51F8043B66
:104BD00040F8043B08BF7047D20728BF31F8023BBA
:104BE00048BF11F8012B28BF20F8023B48BF00F84E
:104BF000012B7047704770477047754600F02CF8DE
:104C0000AE4605006946534620F00700854618B0B9
:104C100020B5FDF70BFABDE820404FF000064FF03D
:104C200000074FF000084FF0000B21F00701AC46E1
:104C3000ACE8C009ACE8C009ACE8C009ACE8C00900
:104C40008D46704710B50446AFF300802046BDE89E
:104C50001040FBF7E8BA000000487047D41D002060
:104C600001491820ABBEFEE7260002007047000095
:104C70008B2D00088F2D0008D32D0008172E00085B
:104C8000412E0008E92E0008132F00083D2F0008D0
:104C9000672F0008912F00086B2E0008952E000842
:104CA000BF2E0008FF2F00082930000855300008EB
:104CB000D04C0008000000208C0A00008C01000885
:104CC000DC4F00088C0A0020AC190000F00100083D
:104CD00012000120050102030404500E0607080912
:104CE0000204060800A24A0400016118E200010360
:104CF00017920001000425FFFF0001C1291005FCE7
:104D0000F368640520070D3F8090943E08200581DC
:104D10009383DE08200582192ABF082005834005F9
:104D20000808200584193E7F0820058580952A08FB
:104D30002005862A7AAA0820058719284F08200509
:104D40008880943A082005898232D10820058A2675
:104D5000790F0820058B192A800820058C8095BAC8
:104D60000820058D6800A10820058E9496D00820A3
:104D7000058F9095BE0852907020059140FA0A0860
:104D800020059241770C0820059341F40B0820057B
:104D90009442B11F0820059542EE0E082005968228
:104DA000301108300497279118200598227C0108BB
:104DB00020059927915F0830049A227B1020059BDB
:104DC00027919F0830049C227F1020059D2791DFAA
:104DD0000830049E227E1030049F1834783004A0DE
:104DE000227F283004A119B0403004A2410088205D
:104DF00005A39096DA082005A4822C4A083004A561
:104E000023A22043A692102005A782325A08340418
:104E1000A81976083404A9822F202005AA4003850A
:104E2000083404AB26EA082005AC2208020843AD8A
:104E300092205405AE18283F7D14053B3FA0924CAC
:104E400014053B3FB03F2B20063B3FA193E60E20CD
:104E500004B13F83152004A292820E13B23F4F206B
:104E6000063B3FA392A70E2004B33F88312004A441
:104E700083490E2004B43F913F2004A59B040E20DB
:104E800004B53FA04D2004A697630E2004B63FA2B0
:104E90005B33A782461004B73FA9701004230100BA
:104EA0008C20053B23BF01701005230319B9152081
:104EB0000522E5002F151705001820063B22C80023
:104EC0002923234820A14323490733E7140742E855
:104ED00015330C043F33E93023330D031C33EA78D8
:104EE000072004EB006062336E0838426F073370AE
:104EF000044D3332003820043300107733F5805BE3
:104F000026B36F20063B22FA003D9A23B400CB3033
:104F100004232F017E20043900201C17F900623081
:104F2000053B23BE02772004B700036932EC23203F
:104F30000522F200302333F880D920040403CF3F48
:104F40001B10124320063B2307F8F8BD33D006C4DC
:104F500033CF60CB42D50742809A4281692EBC1183
:104F60000330053B23B5482332D3E7200522C4068E
:104F700022A12004820340A820048305C09A2004B3
:104F8000287FFFA1322A310FFF22FB4B030DFF4B7D
:104F9000030D364B030E12284B030FE206504B0352
:104FA0000D1044030DFF43030DFF43030D3943036D
:104FB000BE0243030EC81043030E2A004303AD3064
:104FC0000ABC1724562C57445A4849563731563292
:0C4FD000303235303132304623290A00DF
:04000005080001519D
:00000001FF
